:100000000C9458050C949F050C949F050C949F0527
:100010000C949F050C949F050C949F050C949F05D0
:100020000C949F050C949F050C94AC0F0C947E10BF
:100030000C94621E0C949F050C949F050C949F05D4
:100040000C949F050C949F050C949F050C949F05A0
:100050000C949F050C94D61E0C949F050C949F0540
:100060000C949F050C949F050C949F050C949F0580
:100070000C949F050C949F050C949F050C949F0570
:100080000C949F050C949F050C949F050C949F0560
:100090000C949F050C949F050C949F050C949F0550
:1000A0000C949F050C949F050C949F05EB100D116B
:1000B000FB110D11FB1152117511FB11CA11DD114C
:1000C000511551157E157E15D91515160D180D18DB
:1000D0002D160D1828172817E3170D180D18F917E6
:1000E000041607090B0A1D1B06196405141A0815C6
:1000F0001C171E1F202123222E26242D25273012D7
:10010000182F0C13280F0D340E33313638111037D9
:100110002B2C352A5829787B79397A504F515272D5
:100120006C63685680668053020103555880576D92
:100130006E5462595A5B5C5D5E5F6F606174756698
:100140003E3F403C4142774476466B47804365459D
:100150008048494A4B4C3D4D3B4E3A7D7E7C7F73F7
:100160000A0025303862003A2000253032580072EB
:100170002F632030313233343536370A0061646200
:100180005F686F73745F6B62645F726563763A2059
:100190004552524F52282564290A000A002530345E
:1001A00058006164625F686F73745F6B62645F7252
:1001B0006563763A20004552524F523A206D65648D
:1001C0006961206B6579300A004552524F523A20DE
:1001D0006D65646961206B6579310A005D0A0025EF
:1001E000640020002564007C002530325800200087
:1001F00025303258006164625F6D6F7573652072DF
:1002000061773A205B000A00253031366200616474
:10021000625F686F73745F6D6F7573655F7265633E
:10022000763A2000646562756720656E61626C6570
:10023000642E0A005363616E3A20616464723A2549
:10024000642C20726567333A253034580A004166C1
:1002500074657220696E69743A0A00466F756E643F
:100260003A206D65646961206B6579730A00536398
:10027000616E3A20616464723A25642C207265676D
:10028000333A253034580A004265666F726520693A
:100290006E69743A0A005B735D004B6579626F6149
:1002A00072642073746172742E0A00555342206385
:1002B0006F6E666967757265642E0A005B575D0034
:1002C0005B535D005B525D005B445D005B435D0022
:1002D0002E0341004400420020006B0065007900BD
:1002E00062006F00610072006400200063006F0014
:1002F0006E007600650072007400650072000000F8
:100300000E0374002E006D002E006B002E00000006
:100310000403090409027400040100A03209040066
:100320000001030101000921110100012240000721
:1003300005810308000A0904010001030102000904
:100340002111010001224D000705820308000A095E
:1003500004020001030000000921110100012236FE
:10036000000705830308000A0904030002030000D4
:100370000009211101000122220007058403200049
:10038000010705040320000112011001000000080C
:10039000EDFEDB0A0101010200010631FF0974A133
:1003A000010975150026FF00952075088102097660
:1003B000150026FF00952075089102C005010980EF
:1003C000A101850216810026B7001A81002AB70014
:1003D000751095018100C0050C0901A10185031666
:1003E0000100269C021A01002A9C027510950181C9
:1003F00000C005010902A1010901A10005091901B7
:1004000029051500250195057501810295017503E2
:1004100081010501093009311581257F9502750893
:10042000810609381581257F950175088106050C1F
:100430000A38021581257F950175088106C0C0051F
:10044000010906A101050719E029E7150025019515
:1004500008750181029501750881010508190129B6
:10046000059505750191029501750391010507191F
:100470000029FF150026FF00950675088100C00AB7
:10048000002530325820006B6579626F6172645FBD
:100490007265706F72743A20004C45443A202530E2
:1004A00032580A00290A002575002F002575005DC5
:1004B0002800256400200025640020002564002019
:1004C000002564007C0025303258006D6F7573651F
:1004D0006B6579205B62746E7C7820792076206869
:1004E0005D287265702F61636C293A205B006D6B2B
:1004F0005F776865656C5F74696D655F746F5F6D6C
:100500006178203D2025640A006D6B5F7768656522
:100510006C5F6D61785F7370656564203D20256454
:100520000A006D6B5F74696D655F746F5F6D6178F4
:10053000203D2025640A006D6B5F6D61785F7370EC
:10054000656564203D2025640A006D6B5F696E74EB
:10055000657276616C203D2025640A006D6B5F64D6
:10056000656C6179203D2025640A006D6B5F7768BA
:1005700065656C5F74696D655F746F5F6D61782030
:100580003D2025640A006D6B5F776865656C5F6D63
:1005900061785F7370656564203D2025640A006D95
:1005A0006B5F74696D655F746F5F6D6178203D206E
:1005B00025640A006D6B5F6D61785F7370656564BB
:1005C000203D2025640A006D6B5F696E746572764C
:1005D000616C203D2025640A006D6B5F64656C6171
:1005E00079203D2025640A000A00257500363A204E
:1005F000776865656C5F74696D655F746F5F6D6169
:10060000783A20000A00257500353A20776865653C
:100610006C5F6D61785F73706565643A20000A00F5
:10062000257500343A2074696D655F746F5F6D6184
:10063000783A20000A00257500333A206D61785F12
:1006400073706565643A20000A00257500323A200F
:10065000696E74657276616C286D73293A20000AA0
:1006600000257500313A2064656C6179282A3130A3
:100670006D73293A20000A092D2056616C75657347
:10068000202D0A004D3E004D25643E20003F0073A2
:1006900065742064656661756C740A00433E2000D1
:1006A00077686572652064656C74613A2063757261
:1006B000736F723D25642C20776865656C3D2564F9
:1006C0000A53656520687474703A2F2F656E2E7713
:1006D000696B6970656469612E6F72672F77696BEA
:1006E000692F4D6F7573655F6B6579730A000A0931
:1006F0002D204D6F7573656B6579202D0A45534329
:100700002F713A09717569740A313A0964656C612F
:1007100079282A31306D73290A323A09696E746575
:100720007276616C286D73290A333A096D61785FBE
:1007300073706565640A343A0974696D655F746F36
:100740005F6D61780A353A09776865656C5F6D6140
:10075000785F73706565640A363A09776865656C19
:100760005F74696D655F746F5F6D61780A0A703AD6
:10077000097072696E742076616C7565730A643AEB
:10078000097365742064656661756C74730A7570AD
:100790003A092B310A646F776E3A092D310A706776
:1007A00075703A092B31300A7067646F776E3A09B9
:1007B0002D31300A0A7370656564203D2064656CD4
:1007C0007461202A206D61785F7370656564202AEA
:1007D0002028726570656174202F2074696D655FD3
:1007E000746F5F6D6178290A003F004D3E20004321
:1007F0003E20004C25640A000A092D20436F6E73C9
:100800006F6C65202D0A4553432F713A0971756944
:10081000740A6D3A096D6F7573656B65790A000A24
:10082000092D204D61676963202D0A643A096465CA
:100830006275670A783A096465627567206D61744C
:100840007269780A6B3A096465627567206B65792D
:10085000626F6172640A6D3A096465627567206D42
:100860006F7573650A763A0976657273696F6E0AF9
:10087000733A097374617475730A633A09636F6E2E
:10088000736F6C65206D6F64650A302D343A096CA6
:1008900061796572302D34284631302D4634290A6D
:1008A000506175733A09626F6F746C6F6164657241
:1008B0000A003F0074696D65725F7265616433326E
:1008C00028293A202530346C580A006B6579626F0C
:1008D0006172645F69646C653A2025580A006B6533
:1008E00079626F6172645F70726F746F636F6C3A7C
:1008F0002025580A00686F73745F6B6579626F61B9
:1009000072645F6C65647328293A2025580A000ACE
:10091000092D20537461747573202D0A00474343D9
:100920003A20342E392E32204156522D4C49424322
:100930003A20312E382E3073766E204156525F4168
:100940005243483A20617672350A004F5054494F5D
:100950004E533A204C554641204D4F5553454B453B
:10096000592045585452414B455920434F4E534FFF
:100970004C4520434F4D4D414E44204B45594D4130
:10098000505F53454354494F4E20343039360A00A6
:100990004255494C443A2033306131666431202855
:1009A00031303A33303A34372053657020323920B1
:1009B00032303136290A005649443A2030784645CB
:1009C000454428742E6D2E6B2E29205049443A2020
:1009D00030783041444228414442206B6579626F4F
:1009E00061726420636F6E76657274657229205639
:1009F00045523A203078303130310A004445534373
:100A00003A20636F6E7665727420414442206B65B4
:100A100079626F61726420746F205553420A000A34
:100A2000092D2056657273696F6E202D0A000A6DBC
:100A30006F7573653A206F66660A000A6D6F75738D
:100A4000653A206F6E0A000A6B6579626F617264A5
:100A50003A206F66660A000A6B6579626F6172649C
:100A60003A206F6E0A000A6D61747269783A206FDD
:100A700066660A000A6D61747269783A206F6E0AC0
:100A8000000A64656275673A206F6E0A000A646541
:100A90006275673A206F66660A000A0A626F6F74B1
:100AA0006C6F616465722E2E2E2000433E20000084
:100AB00011241FBECFEFDAE0DEBFCDBF04B603FEC8
:100AC00027C08091DC019091DD01A091DE01B09101
:100AD000DF018730904BA740B04BD1F41092DC017E
:100AE0001092DD011092DE011092DF0114BE84B776
:100AF000877F84BF0FB6F894A895809160008861C5
:100B000080936000109260000FBEE0E0F8E309956A
:100B100011E0A0E0B1E0EEE7FEE402C005900D9226
:100B2000A433B107D9F721E0A4E3B1E001C01D92DD
:100B3000AC3DB207E1F70E94DB0C0C943D270C940E
:100B40000000FF93EF93E0913401F091350130976D
:100B500009F00995EF91FF910895FC01859180308E
:100B600011F0EFDFFBCF0895FF27E0E230E247FF0F
:100B70000CC0419597FF09C0EDE260957095809596
:100B80009095611D711D811D911D27FF02C021954A
:100B900030E350E2AA27660F771F881F991FAA1F0C
:100BA000A41710F0A41B63955A95A9F7AA3008F072
:100BB000A95FA05DAF93F39561157105810591055E
:100BC00041F7ED3211F4EF93F395F21718F43F93D8
:100BD000F395FBCF8F91B5DFFA95E1F70895E99191
:100BE000F9918591803021F0853219F0AADFF9CF93
:100BF000089520E0E89455915532C1F3503311F433
:100C0000689455915A3348F4505390F3220F022EB2
:100C1000220F220F200D250FF4CF0EF4219589917C
:100C20009991533619F3533729F1533559F1BC01D2
:100C300088279927E8945C3621F4899199916894E2
:100C40005591543639F446EF7EF077FF0DC08FEFA3
:100C50009FEF0AC055374AE039F0583540E121F09E
:100C6000523642E009F00895FF93EF937DDFEF9154
:100C7000FF91B7CFFF93EF93FC0181918030B9F3DF
:100C800060DFFBCFFF93EF9368DFF1CFDF93CF936C
:100C9000CDB7DEB72596A3DFCF91DF910895282F3A
:100CA0002770E82FE695E695E695EF70F0E0E95CB1
:100CB000FE4F87FF0AC081E090E001C0880F2A95AF
:100CC000EAF780959081892308C081E090E001C017
:100CD000880F2A95EAF79081892B808381E08093A1
:100CE0004C0108950F931F93CF93DF93569A5E9A0A
:100CF0000E94BF092FEF87EA91E621508040904083
:100D0000E1F700C0000088E892E09F938F930E9473
:100D100046060F900F90C1E0D0E00EE612E063E0CF
:100D20008C2F0E94C309009771F09F938F93DF93DC
:100D3000CF931F930F930E9446060F900F900F9032
:100D40000F900F900F909FEF29EF80E0915020407F
:100D50008040E1F700C000002196C031D105F9F6CE
:100D600063E082E00E94C3098131910511F170F4C2
:100D700087309105F1F020F404970297F0F419C040
:100D800089309105B1F00D97C1F413C08D319105F3
:100D900081F030F48431910561F0499771F409C014
:100DA000843C910531F0873C910519F0813C910517
:100DB00021F481E080934D0102C010924D0163E067
:100DC00087E00E94C30991E0823009F090E090939F
:100DD0004E01992341F08BE592E09F938F930E94FF
:100DE00046060F900F9023E042E063E082E00E940D
:100DF000430A8EE492E09F938F930E9446060F90E1
:100E00000F90C1E0D0E004E312E063E08C2F0E9479
:100E1000C309009771F09F938F93DF93CF931F9334
:100E20000F930E9446060F900F900F900F900F9017
:100E30000F908FEF99EF20E0815090402040E1F734
:100E400000C000002196C031D105F9F6E7E3F1E0DA
:100E500080E18E0F11928E13FDCF0E9418120E9416
:100E600066098091BE0181608093BE0184E292E0B8
:100E70000E94AD05569A5E98DF91CF911F910F9118
:100E80000895CF93DF938FE79BEB0197F1F700C0B5
:100E900000000E943F0AEC01009711F481E0C3C0FA
:100EA00097FD05C080914701816080934701D7FF7E
:100EB00005C0809147018E7F809347012D2F3327F6
:100EC0002F733327BE016F737727C6FF02C06054AC
:100ED0007109D6FF02C02054310940913601042E19
:100EE000000C550B649FC001659F900D749F900D81
:100EF000112481386FEF960714F481E89FEF9195E4
:100F00008195910981386FEF960714F481E89FEF7E
:100F1000819580934801249FC001259F900D349FA7
:100F2000900D112481382FEF920714F481E89FEF80
:100F300091958195910981386FEF960714F481E8B6
:100F40009FEF8195809349018091BE0183FF60C02E
:100F50008EE092E00E94AD05DF93CF9388E092E0AF
:100F60009F938F930E94460686E092E00E94AD0513
:100F700085EF91E00E94AD0580913601282F082E63
:100F8000000C330B3F938F9380EF91E09F938F93EF
:100F90000E9446068EEE91E00E94AD0580914701C9
:100FA0001F928F9389EE91E09F938F930E94460644
:100FB00087EE91E00E94AD0580914801282F082E10
:100FC000000C330B3F938F9384EE91E09F938F93AC
:100FD0000E94460682EE91E00E94AD058091490193
:100FE000282F082E000C330B3F938F938FED91E049
:100FF0009F938F930E9446068CED91E00E94AD0571
:101000008DB79EB744960FB6F8949EBF0FBE8DBFA6
:1010100087E491E00E946D128091360191E0883062
:101020000CF090E0890F80933601DF91CF91089505
:101030001F93CF93DF9310924C01C0910001D09188
:1010400001018FEF9FEF9093010180930001CF3F4B
:101050008FEFD80709F06AC08FE79BEB0197F1F794
:1010600000C0000082E00E943C0AEC01892B09F0DC
:101070005DC080914E01882309F458C087E00E942A
:101080003C0A009709F452C09C012F773327223085
:101090003105A1F048F42115310569F02130310501
:1010A00099F480788A641AC02330310551F02F37C3
:1010B0003105A1F009C08078826410C0807889640D
:1010C0000DC0807888640AC089EC91E09F938F936B
:1010D0000E9446060F900F9081E18FC0292F332781
:1010E0002F7733272130310579F050F02230310548
:1010F00079F02330310581F4EC01D078D86416C042
:10110000EC01D078D26412C0EC01D078DA640EC061
:10111000EC01D078D9640AC086EB91E09F938F935D
:101120000E9446060F900F9080E167C08091BE013B
:1011300081FF18C0209709F45DC082EA91E00E9407
:10114000AD05DF93CF938DE991E09F938F930E943C
:1011500046068BE991E00E94AD050F900F900F902D
:101160000F9003C0209709F445C0CF379FE7D907F8
:1011700011F48FE705C0CF3F8FEFD80721F48FEF31
:101180000E944F0639C02D2F3327822F1C2F2F3F4F
:10119000310581F4DF93CF938DE791E09F938F9397
:1011A0000E9446060E9472060F900F900F900F90BB
:1011B0008C2F23C090914D01992381F0A9014F7785
:1011C00055274233510521F42078822F8A6006C0CA
:1011D0004A30510519F42078822F82630E944F060D
:1011E0001F3F51F0DC2FCC27CF6FD0930101C0936C
:1011F000000102C080E001C081E0DF91CF911F912A
:101200000895E82FF0E0E95CFE4F2081822F90E006
:1012100021E030E002C0220F331F6A95E2F7282355
:10122000392381E0232B09F480E00895E82FF0E0D2
:10123000E95CFE4F80810895CF92DF92EF92FF929A
:101240000F931F93CF93DF938091BE0181FF35C031
:101250008FE691E00E94AD0587E3E82E81E0F82E4D
:10126000C0E0D0E09AE6C92E91E0D92E02E611E066
:10127000DF93CF93DF92CF920E94460687E691E0FC
:101280000E94AD05F70181917F010E94F71D1F9219
:101290008F931F930F930E94460680E691E00E9471
:1012A000AD0521968DB79EB708960FB6F8949EBFF0
:1012B0000FBE8DBFC031D105D9F6DF91CF911F91FF
:1012C0000F91FF90EF90DF90CF900895682F609579
:1012D00082E00C947D0A509A83E091E00197F1F747
:1012E00000C0000050989AEB9A95F1F700C008955D
:1012F000509A8AEB8A95F1F700C0509883E091E00C
:101300000197F1F700C000000895EF92FF920F934C
:101310001F93CF93DF93C0E0D0E090E8E92EF12C4B
:10132000082F10E0C7010C2E02C0959587950A94EE
:10133000E2F780239123892B19F00E94780902C0DB
:101340000E946B092196C830D10561F7DF91CF91DA
:101350001F910F91FF90EF900895489B06C023E0E6
:101360002A95F1F700000197C1F70895489906C042
:1013700023E02A95F1F700000197C1F708955898E6
:10138000509808950895CF92DF92EF92FF920F93B5
:101390001F93CF93DF931F92CDB7DEB7182FF8942A
:1013A000509A83EF9BE00197F1F700C0000069833A
:1013B0000E94780969816C6020E1129FC0011124AC
:1013C000862B0E9485090E946B0984EF91E00E94A0
:1013D000B609892B21F4789482EE9FEF43C084EF05
:1013E00091E00E94AD09009711F478943BC011E19F
:1013F000C12CD12C02E882E890E00E94B6097C0161
:10140000882351F199270E94AD09882329F1CC0C3A
:10141000DD1C902F9E19E81A9E1518F46894C0F8E8
:1014200006C0113121F478948CEE9FEF1BC011504F
:1014300011F78FE591E00E94B609892B21F4789489
:101440008BEE9FEF0FC08BE590E00E94AD09892BDA
:10145000B1F77894C60106C07894812F90E09195F9
:10146000819591090F90DF91CF911F910F91FF907E
:10147000EF90DF90CF90089560E00C94C30960E096
:1014800083E00C94C3091F93CF93DF9300D01F9286
:10149000CDB7DEB7182FF894509A83EF9BE00197F1
:1014A000F1F700C000002B834A8369830E9478090A
:1014B0006981686030E1139FC0011124862B0E946E
:1014C00085090E946B098FE193E00197F1F700C055
:1014D00000000E9478094A81842F0E9485092B818F
:1014E000822F0E9485090E946B0978940F900F90BB
:1014F0000F90DF91CF911F910895262F277040E024
:1015000062E00C94430A80915A0108959FB7F894C1
:10151000109251019FBF9091D301943009F057C0B0
:101520009091E9009F703091EC00232F217030FDE5
:1015300020E8922B24E02093E9002091EB0020FF8B
:1015400043C02091EE0027FF3FC020914F0122238E
:1015500021F02091E80025FF37C010924F0126E0CE
:101560003091E80035FD15C03091D301343061F57C
:101570003091EB0035FD28C0215021F481E08093AB
:101580004F0122C0EFE9FFE03197F1F700C0000002
:10159000E7CF8093F1008091E80085FD0AC080913B
:1015A000E80080FFFCCF8091E8008E778093E80010
:1015B00006C08FB7F89421E0209351018FBF9F7030
:1015C0009093E90080E008959F709093E9008FEF79
:1015D0000895CF93DF9300D01F92CDB7DEB79C0163
:1015E0008091D301843019F593E099833B832A835A
:1015F0009093E9008FEF9091E800815095FD06C02F
:1016000095ED9A95F1F700008111F5CF8091E800F2
:1016100085FF0DC040E050E063E070E0CE01019630
:101620000E949C0D8091E8008E778093E8000F90D7
:101630000F900F90DF91CF910895CF93DF9300D05B
:101640001F92CDB7DEB72091D301243021F522E0DF
:1016500029839B838A8383E08093E9008FEF9091B5
:10166000E800815095FD06C095ED9A95F1F70000D0
:101670008111F5CF8091E80085FF0DC040E050E07A
:1016800063E070E0CE0101960E949C0D8091E8001D
:101690008E778093E8000F900F900F90DF91CF919D
:1016A00008952091D3012430F1F422E02093E90041
:1016B0002FEF3091E800215035FD06C035ED3A9509
:1016C000F1F700002111F5CF2091E80025FF0BC0B4
:1016D00040E050E065E070E00E949C0D8091E800E1
:1016E0008E778093E8000895CF93DF932091D30104
:1016F000243039F521E02093E9002FEF3091E80004
:10170000215035FD06C035ED3A95F1F70000211165
:10171000F5CF2091E80025FF14C0EC0140E050E037
:1017200068E070E00E949C0D8091E8008E778093C5
:10173000E80088E0FE01A2E5B1E001900D928A95F3
:10174000E1F7DF91CF9108958CEC92E00E94AD0516
:101750008091D201811109C00E94310F0E948E0F29
:101760008091E20084608093E200089588EC92E02A
:101770000E94AD051092D201089584EC92E00C9481
:10178000AD05209150012F5F822F62E30E94032755
:10179000992319F0209350010895109250018091DF
:1017A0005101882371F18091D301843041F58091FA
:1017B000E9008F702091EC00922F917020FD90E84D
:1017C000892B94E09093E9009091EB0090FF14C076
:1017D0009091EE0097FF10C09091E80095FF03C034
:1017E0001092F100F9CF9091E80090FF05C0909120
:1017F000E8009E779093E8008F708093E900109244
:101800005101089542E061EC81E00E94AB0E42E09C
:1018100061EC82E00E94AB0E42E061EC83E00E944A
:10182000AB0E42E261EC84E00C94AB0E8091D501EA
:10183000833009F453C030F4813071F0823009F400
:101840008CC008958A3009F478C08B3009F45EC0EA
:10185000893009F09AC020C08091D401813A09F002
:1018600094C08091E800877F8093E8008091D80140
:101870009091D901892B21F468E082E591E003C0C1
:1018800060E080E090E070E00E94E70D8091E80069
:101890008B778093E80008958091D401813209F01C
:1018A00074C08091D8019091D901892B09F06DC045
:1018B0008091E800877F8093E8008091E80082FDB6
:1018C00005C08091D3018111F8CF5FC08091F100F4
:1018D00080935A018091E8008B7753C08091D401A6
:1018E000813A09F052C08091D8019091D901892B99
:1018F00009F04BC08091E800877F8093E8008091D9
:10190000E80080FFFCCF80910C0136C08091D401AB
:101910008132D9F58091D8019091D901892BA9F50F
:101920008091E800877F8093E8000E94E00E80911C
:10193000D60180930C010C942E188091D401813231
:1019400021F58091E800877F8093E8000E94E00EF7
:101950008091D70180935B0108958091D401813AF1
:10196000A1F48091E800877F8093E8008091E800EF
:1019700080FFFCCF80915B018093F1008091E800B3
:101980008E778093E8000C94E00E089508950895F2
:10199000089580EC92E00E94AD050C94C80C0E9462
:1019A000211E8091D101882329F00E944C1E8111B3
:1019B0000C94860D089584B7877F84BF0FB6F89482
:1019C000A89580916000886180936000109260000B
:1019D0000FBE90E080E80FB6F8948093610090937A
:1019E00061000FBE0E94C60C0E94A5120E94310F1A
:1019F0000E948E0F8091E20084608093E20086E86E
:101A00009AE00E94F21D78948091D3018430E1F72E
:101A10008BEA92E00E94AD050E94A71282E091E05D
:101A20000E9413128AE992E00E94AD050E94C70C41
:101A30008091D301853039F486E992E00E94AD05AA
:101A40000E94CF0CF5CF0E94AD12F2CF0C94601E15
:101A50008CEB92E00E94AD050C94260D292F3327C4
:101A600023303105C9F064F42130310581F0223092
:101A7000310509F043C084E790E024E133E042C03F
:101A800021323105F1F02232310541F137C082E1D6
:101A900090E028E833E036C099278130910541F085
:101AA0008230910541F0892B49F5E0E1F3E005C072
:101AB000E0E0F3E002C0E0EDF2E0849190E09F010D
:101AC00021C06430D8F4E62FF0E0EE0FFF1FEF5D89
:101AD000FE4F2081318189E090E014C0643070F4C1
:101AE00070E0FB01EE0FFF1FE75EFE4F20813181AA
:101AF000FB01EB5EFE4F808190E004C080E090E04F
:101B000020E030E0FA0131832083089580E189BD2F
:101B100082E189BD09B400FEFDCF8091D8008F7DA0
:101B20008093D8008091E00082608093E0008091F3
:101B3000E00081FDFCCF0895CF92DF92EF92FF92FB
:101B40000F931F93CF93DF93EC018B016A010E94E7
:101B5000FF0E811133C0C114D10439F0F601808128
:101B60009181081B190BC80FD91FE12CF12C01150D
:101B7000110519F18091E80085FD16C08091E800FB
:101B80008E778093E800C114D10449F0F60180817A
:101B90009181E80EF91EF182E08285E00FC00E947B
:101BA000FF0E882321F30AC089918093F100015030
:101BB0001109FFEFEF1AFF0ADACF80E0DF91CF9132
:101BC0001F910F91FF90EF90DF90CF90089520919B
:101BD000DA013091DB012617370748F061157105EE
:101BE00039F42091E8002E772093E80001C0B90174
:101BF00040E061157105A9F12091D301222309F478
:101C000043C0253009F442C02091E80023FD40C0C4
:101C10002091E80022FD32C02091E80020FFE9CFAA
:101C20004091F3002091F20030E0342BFC01CF0111
:101C30006115710559F02830310540F48191809388
:101C4000F100615071092F5F3F4FF1CF41E0283023
:101C5000310509F040E02091E8002E772093E8005C
:101C6000C8CF4111C9CF0AC08091D301882361F048
:101C7000853061F08091E80083FD0AC08091E80022
:101C800082FFF2CF80E0089582E0089583E0089516
:101C900081E008952091DA013091DB0126173707A2
:101CA00048F06115710539F42091E8002E772093F2
:101CB000E80001C0B901FC0120E06115710591F156
:101CC0008091D301882309F440C0853009F43FC0D6
:101CD0008091E80083FD3DC08091E80082FD2FC027
:101CE0008091E80080FFE9CF2091F3008091F2001D
:101CF00090E0922B6115710559F08830910540F400
:101D000024912093F1003196615071090196F2CF30
:101D100021E0089709F020E08091E8008E77809319
:101D2000E800CBCF2111CCCF0AC08091D30188230A
:101D300061F0853061F08091E80083FD0AC08091F8
:101D4000E80082FFF2CF80E0089582E0089583E00A
:101D5000089581E00895982F973058F59093E90001
:101D6000981739F07091EC002091ED005091F0003F
:101D700003C0242F762F50E021FF19C03091EB00D3
:101D80003E7F3093EB003091ED003D7F3093ED00CE
:101D90003091EB0031603093EB007093EC002093B6
:101DA000ED005093F0002091EE0027FF07C09F5FE9
:101DB000D3CF8F708093E90081E0089580E008958B
:101DC0008091D40187FF11C08091E80082FD05C099
:101DD0008091D3018111F8CF11C08091E8008B77F9
:101DE0000BC08091D301882349F08091E80080FFE7
:101DF000F8CF8091E8008E778093E80008952091D5
:101E0000E4003091E50095E64091EC00842F81706C
:101E100040FF22C08091E80080FD1CC08091D3016A
:101E2000882391F0853091F08091EB0085FD10C002
:101E30004091E4005091E5004217530729F39A01BD
:101E4000915011F784E0089582E0089583E00895A9
:101E500081E0089580E008954091E80042FFDECFE0
:101E600008950E949F0F0E94A70FE0EEF0E080818E
:101E700081608083E8EDF0E080818F77808319BCFA
:101E8000A7EDB0E08C918E7F8C9380818F7E8083D4
:101E90001092D20108950F931F93CF93DF930E9466
:101EA0009F0F0E94A70FC8EDD0E088818F778883AD
:101EB00088818068888388818F7D888319BC10928F
:101EC000D3011092CF011092D1011092D00100EEF7
:101ED00010E0F80180818B7F808388818160888316
:101EE00042E060E080E00E94AB0EE1EEF0E0808135
:101EF0008E7F8083E2EEF0E080818160808380814C
:101F000088608083F80180818E7F808388818061F2
:101F10008883DF91CF911F910F910895E8EDF0E054
:101F200080818F7E8083E7EDF0E080818160808317
:101F300084E082BF81E08093D2010C944B0FE8EDE6
:101F4000F0E080818E7F80831092E20008951092ED
:101F5000DA001092E10008951F920F920FB60F92CF
:101F600011242F933F934F935F936F937F938F939E
:101F70009F93AF93BF93EF93FF938091E10082FF14
:101F80000BC08091E20082FF07C08091E1008B7F4F
:101F90008093E1000E94C10B8091DA0080FF1FC096
:101FA0008091D80080FF1BC08091DA008E7F8093E3
:101FB000DA008091D90080FF0DC080E189BD82E107
:101FC00089BD09B400FEFDCF81E08093D3010E945A
:101FD000A40B05C019BC1092D3010E94B60B8091CE
:101FE000E10080FF19C08091E20080FF15C0809160
:101FF000E2008E7F8093E2008091E2008061809316
:10200000E2008091D80080628093D80019BC85E0FE
:102010008093D3010E94C90C8091E10084FF30C0FD
:102020008091E20084FF2CC080E189BD82E189BDFE
:1020300009B400FEFDCF8091D8008F7D8093D80039
:102040008091E1008F7E8093E1008091E2008F7E9D
:102050008093E2008091E20081608093E2008091B1
:10206000CF01882311F084E007C08091E30087FD51
:1020700002C081E001C083E08093D3010E94280D5B
:102080008091E10083FF29C08091E20083FF25C099
:102090008091E100877F8093E10082E08093D3010B
:1020A0001092CF018091E1008E7F8093E1008091BA
:1020B000E2008E7F8093E2008091E2008061809355
:1020C000E20042E060E080E00E94AB0E8091F00010
:1020D00088608093F0000E94BD0BFF91EF91BF914B
:1020E000AF919F918F917F916F915F914F913F91B0
:1020F0002F910F900FBE0F901F9018951F920F9267
:102100000FB60F9211242F933F934F935F936F93CA
:102110007F938F939F93AF93BF93CF93DF93EF936F
:10212000FF93C091E900CF708091EC00D82FD1705F
:1021300080FDD0E81092E9008091F000877F8093C5
:10214000F00078940E94C2101092E9008091F00093
:1021500088608093F000CD2BCF70C093E900FF9191
:10216000EF91DF91CF91BF91AF919F918F917F912F
:102170006F915F914F913F912F910F900FBE0F90F4
:102180001F9018951F93CF93DF93CDB7DEB7AA9713
:102190000FB6F894DEBF0FBECDBFE4EDF1E088E0EE
:1021A0008E0F9091F10091938E13FBCF0E94160C2D
:1021B0008091E80083FF1FC18091D4019091D501E7
:1021C000492F50E04A30510508F015C1FA01EA5A8A
:1021D000FF4F0C942327803881F0823809F00BC11F
:1021E0008091D8018F708093E9008091EB0085FB8E
:1021F000882780F91092E90006C08091D001909163
:10220000D101911182609091E800977F9093E8004E
:102210008093F1001092F100C8C0282F2D7F09F0A3
:10222000EAC0882319F0823061F0E5C08091D601C0
:10223000813009F0E0C0933009F080E08093D10153
:102240002BC08091D601811127C08091D8018F7059
:1022500009F4D1C08093E9002091EB0020FF1CC05D
:10226000933021F48091EB00806214C09091EB00D8
:1022700090619093EB0021E030E0A90102C0440F8F
:10228000551F8A95E2F74093EA001092EA00809188
:10229000EB0088608093EB001092E9008091E800E9
:1022A000877F86C08111A7C01091D6011F778091CA
:1022B000E3008078812B8093E3008091E800877FA2
:1022C0008093E8000E94E00E8091E80080FFFCCF40
:1022D0008091E30080688093E300111102C082E0E6
:1022E00001C083E08093D30186C08058823008F01B
:1022F00082C08091D6019091D7018C3D53E0950723
:1023000079F583E08A838AE289834FB7F894DE0106
:10231000139620E03EE051E2E32FF0E050935700A7
:10232000E49120FF03C0E295EF703F5FEF708E2FC6
:1023300090E0EA3010F0C79601C0C0968D939D934F
:102340002F5F243149F74FBF8091E800877F80934A
:10235000E8006AE270E0CE0101960E94E70D14C029
:10236000AE014F5F5F4F6091D8010E942E0DBC01FE
:10237000892B09F440C09091E800977F9093E80082
:1023800089819A810E944A0E8091E8008B77809320
:10239000E80031C0803879F58091E800877F80932C
:1023A000E8008091CF018093F1008091E8008E7762
:1023B0008093E8000E94E00E1EC081111CC0909125
:1023C000D6019230C0F48091E800877F8093E800C6
:1023D0009093CF010E94E00E8091CF01811106C041
:1023E0008091E30087FD02C081E001C084E080931A
:1023F000D3010E94020C8091E80083FF0AC0809103
:10240000E800877F8093E8008091EB0080628093F2
:10241000EB00AA960FB6F894DEBF0FBECDBFDF91DA
:10242000CF911F9108959093610180936001089569
:10243000E0916001F0916101309721F00190F0810D
:10244000E02D099480E00895EF92FF920F931F937F
:10245000CF93DF93E0916001F09161013097B1F18A
:102460008C010280F381E02D09958091BE0182FFED
:102470002DC080FF04C087E894E00E94AD05E8010C
:1024800018E081E8E82E84E0F82E8091BE0180FFFC
:102490000BC088811F928F93FF92EF920E94460695
:1024A0000F900F900F900F90115021961111EDCFBA
:1024B0008091BE0180FF0AC08FE794E0DF91CF9149
:1024C0001F910F91FF90EF900C94AD05DF91CF918C
:1024D0001F910F91FF90EF900895E0916001F091AE
:1024E0006101309721F00480F581E02D0994089571
:1024F00020915E0130915F018217930771F09093F4
:102500005F0180935E01E0916001F091610130977D
:1025100021F00680F781E02D0994089520915C0157
:1025200030915D018217930771F090935D01809364
:102530005C01E0916001F0916101309721F000842D
:10254000F185E02D0994089508950C94A4120E9439
:102550008B1E0E9472060C94C209CF92DF92EF92FA
:10256000FF920F931F93CF93DF9300D000D000D042
:10257000CDB7DEB70E94180883E6C82E81E0D82EBA
:1025800000E010E0E02E802F0E941609F601419134
:102590006F01F42EF826B1F40F5F1F4F00311105C3
:1025A00089F78FEF89838A831B820E94941E816042
:1025B000782F9D838C8349815A816B818D810E9404
:1025C0006E1347C09091BE0191FF04C08E830E949C
:1025D0001C098E8120E030E04F2D50E0922FBA018F
:1025E000022E02C0759567950A94E2F760FF2BC032
:1025F0002983EA8221E030E0690102C0CC0CDD1CB5
:102600009A95E2F790E08C219D21892B09F420E036
:102610002B830E94941E8160782F9D838C83498137
:102620005A816B818D810E946E1349815A816B8121
:102630007C818D810E940E1EF801ED59FE4F808134
:10264000C826C08206C02F5F3F4F2830310531F6C3
:10265000A3CF0E940D1E0E9455210E944107109198
:1026600062010E941812181741F10E9418128093FB
:1026700062019091BE0192FF0EC090FF0CC01F92AC
:102680008F9389E994E09F938F930E9446060F9061
:102690000F900F900F908091620126960FB6F894DC
:1026A000DEBF0FBECDBFDF91CF911F910F91FF9085
:1026B000EF90DF90CF900C941F1E26960FB6F894E3
:1026C000DEBF0FBECDBFDF91CF911F910F91FF9065
:1026D000EF90DF90CF9008950C946609CF93DF932D
:1026E000CDB7DEB72B970FB6F894DEBF0FBECDBFC8
:1026F000942F4F83252F588769877A878B874A8540
:102700005B85452B21F02F3F09F59F3FF9F4DE0152
:10271000119686E0FD0111928A95E9F785E0FE01A8
:10272000379601900D928A95E1F749815A816B8124
:102730007C818D819E810E94C81A2B960FB6F894D9
:10274000DEBF0FBECDBFDF91CF9108954F81588579
:1027500069857A858B850E940E1ED9CFCF938823F9
:1027600009F4E8C0C82F8238A1F40E94181281FD34
:10277000E1C089E30E94531D0E94CC1D2FEF81EE22
:1027800094E0215080409040E1F700C0000089E3D0
:1027900015C08338C1F40E94181280FDCBC083E5B8
:1027A0000E94531D0E94CC1D2FEF81EE94E021501A
:1027B00080409040E1F700C0000083E50E94701D5A
:1027C000CF910C94CC1D8438A1F40E94181282FD84
:1027D000B1C087E40E94531D0E94CC1D2FEF81EEF3
:1027E00094E0215080409040E1F700C0000087E471
:1027F000E5CF8CEF8C0F813A48F48C2F0E947F2418
:10280000811198C08C2F0E94531DDACF80E28C0F6B
:10281000883048F4C77081E001C0880FCA95EAF794
:102820000E94921DCDCF8BE58C0F833078F4C53A92
:1028300029F0C63A31F083E890E005C081E890E0E5
:1028400002C082E890E0CF910C94781288E58C0F5A
:10285000853108F06FC0C83A61F1C93A69F1CA3AE6
:1028600071F1CB3A79F1CC3A81F1CD3A89F1CE3A96
:1028700091F1CF3A99F1C13BA1F1C03BA9F1C23B23
:10288000B1F1C33BB9F1C43BC1F1C53BC9F1C63B92
:10289000D1F1C73BD9F1C83BE1F1C93BE9F1CA3BF2
:1028A000F1F1CB3BF9F1CC3B09F43FC080E090E083
:1028B0003EC082EE90E03BC089EE90E038C08AEEE8
:1028C00090E035C085EB90E032C086EB90E02FC001
:1028D00083EB90E02CC084EB90E029C087EB90E084
:1028E00026C08CEC90E023C08DEC90E020C083E803
:1028F00091E01DC08AE891E01AC082E991E017C01A
:1029000084E991E014C081E292E011C083E292E098
:102910000EC084E292E00BC085E292E008C086E23D
:1029200092E005C087E292E002C08AE292E0CF9195
:102930000C948E12CF910895882309F466C08238D2
:10294000A1F40E94181281FF60C089E30E94531D08
:102950000E94CC1D2FEF81EE94E0215080409040EA
:10296000E1F700C0000089E315C08338B9F40E9484
:10297000181280FF4AC083E50E94531D0E94CC1D9F
:102980002FEF81EE94E0215080409040E1F700C0AD
:10299000000083E50E94701D0C94CC1D8438A1F4C6
:1029A0000E94181282FF31C087E40E94531D0E94CA
:1029B000CC1D2FEF81EE94E0215080409040E1F754
:1029C00000C0000087E4E6CF9CEF980F913A10F327
:1029D00090E2980F983050F4877091E001C0990F01
:1029E0008A95EAF7892F0E94981DD6CF9BE5980F0C
:1029F000933020F480E090E00C947812885A85316E
:102A000020F480E090E00C948E120895882321F049
:102A10000E94921D0C94CC1D0895882321F00E94E1
:102A2000981D0C94CC1D0895CF92DF92EF92FF92E7
:102A30000F931F93CF93DF9300D000D000D0CDB77A
:102A4000DEB725E0FC01DE01119601900D922A957A
:102A5000E1F7FC0140813181F280258122952F70C0
:102A600063817481672B09F4D8C23F3F19F44F3F4B
:102A700009F4D3C26C0149833A8389819A812E83F8
:102A80000E94121D182F092F0E94111D0E94211C47
:102A9000E02FE295EF70F0E0E05AFF4F2E810C94AA
:102AA0002327802F807F902F9F70092F882311F07C
:102AB0000295007FFF2049F0002309F45FC2802FB8
:102AC0000E94A51D0E94CC1D59C2812F0E949C14FA
:102AD000002309F4A2C2802F0E94AB1D26960FB6D8
:102AE000F894DEBF0FBECDBFDF91CF911F910F9144
:102AF000FF90EF90DF90CF900C94CC1D802F807FC3
:102B0000902F9F70092F803211F00295007F1123C2
:102B100019F0113001F129C0FF20A9F0802F2223E4
:102B200049F1213039F526960FB6F894DEBF0FBE75
:102B3000CDBFDF91CF911F910F91FF90EF90DF906C
:102B4000CF900C94B51D222319F0213009F465C2F1
:102B50000E94B81D2CC0FF20E9F0263008F05DC2AD
:102B60000E948F1D802329F022C0FF20F1F0211147
:102B700015C0802F26960FB6F894DEBF0FBECDBFCE
:102B8000DF91CF911F910F91FF90EF90DF90CF9049
:102B90000C940615253008F040C209C0F601858165
:102BA00080FFECC18F708583E4CF2111FBC1802FA2
:102BB00069C1202F26952695237030E02115310517
:102BC00021F021303105C9F028C2FF2021F0812FEA
:102BD000902F937002C080E090E026960FB6F89494
:102BE000DEBF0FBECDBFDF91CF911F910F91FF9040
:102BF000EF90DF90CF900C947812FF2021F0812F7E
:102C0000902F937002C080E090E026960FB6F89463
:102C1000DEBF0FBECDBFDF91CF911F910F91FF900F
:102C2000EF90DF90CF900C948E12812FFF2019F03F
:102C30000E94DB1F02C00E94432026960FB6F89424
:102C4000DEBF0FBECDBFDF91CF911F910F91FF90DF
:102C5000EF90DF90CF900C94C820802F837009F004
:102C600078C0F110DAC1812F829586958770880F20
:102C7000880F912F9F70C92ED12CE12CF12C082E9A
:102C800004C0CC0CDD1CEE1CFF1C0A94D2F714FF10
:102C900012C04FE050E060E070E004C0440F551FE8
:102CA000661F771F8A95D2F7CB01BA0160957095A0
:102CB0008095909503C060E070E0CB01202F2695B1
:102CC00026952370422F50E042305105D1F0433019
:102CD000510559F16C297D298E299F2941305105D3
:102CE00041F126960FB6F894DEBF0FBECDBFDF913F
:102CF000CF911F910F91FF90EF90DF90CF900C94A8
:102D0000361C6C297D298E299F2926960FB6F894AA
:102D1000DEBF0FBECDBFDF91CF911F910F91FF900E
:102D2000EF90DF90CF900C94481C0E94361CC70196
:102D3000B60126960FB6F894DEBF0FBECDBFDF9169
:102D4000CF911F910F91FF90EF90DF90CF900C9457
:102D5000241CFF2019F0802F817001C086958823E4
:102D600009F45BC1812F829586958770880F880F43
:102D7000912F9F70C92ED12CE12CF12C082E04C06C
:102D8000CC0CDD1CEE1CFF1C0A94D2F714FF12C001
:102D90004FE050E060E070E004C0440F551F661F34
:102DA000771F8A95D2F7CB01BA016095709580950F
:102DB000909503C060E070E0CB01202F269526950A
:102DC0002370422F50E042305105D1F0433051057D
:102DD00059F16C297D298E299F294130510541F1F6
:102DE00026960FB6F894DEBF0FBECDBFDF91CF9110
:102DF0001F910F91FF90EF90DF90CF900C94ED1CFE
:102E00006C297D298E299F2926960FB6F894DEBF5E
:102E10000FBECDBFDF91CF911F910F91FF90EF902B
:102E2000DF90CF900C94FF1C0E94ED1CC701B601EF
:102E300026960FB6F894DEBF0FBECDBFDF91CF91BF
:102E40001F910F91FF90EF90DF90CF900C94DB1CBF
:102E5000103F41F118F4103E48F48BC0123F09F4C2
:102E600050C0D8F1133F09F460C083C01F70802F99
:102E70008F71FF2021F00E94741C812F7BCE0E9455
:102E8000951C812F26960FB6F894DEBF0FBECDBFDE
:102E9000DF91CF911F910F91FF90EF90DF90CF9036
:102EA0000C940D15FF20A9F0253008F0B6C0802F36
:102EB0008F7126960FB6F894DEBF0FBECDBFDF919F
:102EC000CF911F910F91FF90EF90DF90CF900C94D6
:102ED000BA1C263008F0A1C0EACFFF20A1F0802F55
:102EE0008F7126960FB6F894DEBF0FBECDBFDF916F
:102EF000CF911F910F91FF90EF90DF90CF900C94A6
:102F0000741CFF2061F3802F8F7126960FB6F89402
:102F1000DEBF0FBECDBFDF91CF911F910F91FF900C
:102F2000EF90DF90CF900C94951CFF2091F0802FB4
:102F30008F7126960FB6F894DEBF0FBECDBFDF911E
:102F4000CF911F910F91FF90EF90DF90CF900C9455
:102F50005F1C26960FB6F894DEBF0FBECDBFDF9183
:102F6000CF911F910F91FF90EF90DF90CF900C9435
:102F70005A1CFF20A1F0222309F4B1CF812F2696FD
:102F80000FB6F894DEBF0FBECDBFDF91CF911F917A
:102F90000F91FF90EF90DF90CF900C94AE1322230F
:102FA00009F4B1CF812F26960FB6F894DEBF0FBE7D
:102FB000CDBFDF91CF911F910F91FF90EF90DF90E8
:102FC000CF900C949C14402F4F70612FC6010E942B
:102FD000551F26960FB6F894DEBF0FBECDBFDF910A
:102FE000CF911F910F91FF90EF90DF90CF900C94B5
:102FF0006C1B402F4F70612FC60126960FB6F894B8
:10300000DEBF0FBECDBFDF91CF911F910F91FF901B
:10301000EF90DF90CF900C94581F26960FB6F8943F
:10302000DEBF0FBECDBFDF91CF911F910F91FF90FB
:10303000EF90DF90CF9008950E94B21D0E94811DF5
:103040000E94CC1D0E94FA210E94C82080E090E0DE
:103050000E94781280E090E00C948E120E94A21DD3
:103060000C941C180E94121D292F22952F7030E0FD
:103070002C3031054CF42A3031056CF422503109E2
:103080002230310588F407C02C30310549F02F304B
:10309000310531F009C0803E48F0803F29F406C078
:1030A00093FB882780F9089580E0089581E00895D2
:1030B000CF93DF9300D000D01F92CDB7DEB70F9033
:1030C0000F900F900F900F90DF91CF910895CF93B5
:1030D000DF9300D000D000D0CDB7DEB726960FB674
:1030E000F894DEBF0FBECDBFDF91CF9108951F933F
:1030F000CF93DF93C091730116E080917401C817DC
:1031000099F0D0E01C9FF0011D9FF00D1124EB58A9
:10311000FE4F4081518162817381848195810E943B
:1031200067182196C770E9CFDF91CF911F9108955D
:103130004091A5015091A6016091A7017091A8014D
:103140008091A9019091AA010C9467188091AA011D
:1031500082958F7009F054C08091A701882309F4EB
:103160004FC080917301A09174016091A50170918D
:10317000A6014091A8015091A901B6E08A1709F46F
:103180003FC090E041155105C1F17F3F11F46F3F01
:10319000A1F1B89FF001B99FF00D1124EB58FE4F3B
:1031A000218172132AC02081621327C0228121113C
:1031B00024C0238134812417350710F421503109AC
:1031C000241B350B283C3105C0F42091AA012F7037
:1031D00020612093AA0126E0289FF001299FF00D8D
:1031E0001124E658FE4F80818F708061808385EACC
:1031F00091E00E9414150C94771801968770BECF49
:103200000895CF92DF92EF92FF920F931F93CF9387
:10321000DF93CDB7DEB762970FB6F894DEBF0FBE6F
:10322000CDBF8C0185E0F801DE011D9601900D9265
:103230008A95E1F7D8014C9111965C9111971296FD
:103240006C9112971396CD90DC9014973091A50154
:103250007091A6018091A8019091A901009709F4AD
:103260006BC17F3F19F43F3F09F466C1E090A701AD
:10327000EE2009F4C0C02091AA01C816D90628F092
:10328000F601E81BF90BCF0104C0809590958C0DD9
:103290009D1DFF24F394883C910578F0F12C207F4C
:1032A00009F0C6C07C2DD98AC88A89890E9458181D
:1032B00085EA91E00E941415B1C0822F807F09F049
:1032C00046C0751314C0341312C0611110C02F70A2
:1032D00020612093AA010E94981885EA91E00E943B
:1032E00014158091AA01D80115968C932EC0CD2873
:1032F00019F15F3F11F44F3FF9F0F62E61111CC038
:10330000809173012091740136E0821709F45AC04C
:1033100090E0389FF001399FF00D1124EB58FE4FDB
:103320007181571306C07081471303C072817111F8
:1033300003C001968770E9CFF62E662309F418C101
:103340008091AA0181608093AA01F12C11C17513AB
:1033500008C0341306C0611104C08091AA01D801CD
:10336000C3C04D875E878D859E856A8B0E9432180B
:103370006A898823E1F16623D1F12091AA01822F85
:1033800082958F7090E0029774F08091A5019091E2
:10339000A60198878F831986DB86CA862C87CE0183
:1033A00007960E94141586E0F801A5EAB1E00190A5
:1033B0000D928A95E1F70E94A6180E949818FF24A2
:1033C000F394D6C04D875E878D859E850E94121D21
:1033D000292F22952F7030E0223031050CF0BCC02F
:1033E0009F7009F0B6C0805E883008F4C1C0C80183
:1033F0000E941415E4CFC816D90608F453C0F6018C
:10340000E81BF90BCF01883C910508F450C0F12C62
:103410007C2DD98AC88A89890E945818E5EAF1E08A
:1034200086E0DF011D928A95E9F70E949818A0C0F6
:10343000751314C0341312C0611110C08091AA0119
:10344000F8018583C8010E94141586E0E5EAF1E0E1
:10345000DF011D928A95E9F7FE2C8AC04D875E87B1
:103460008D859E856A8B0E9432186A89882309F4AB
:10347000BECF662309F4BBCF2091AA01822F82958B
:103480008F7090E002970CF48ECF8091A5019091FF
:10349000A6019A8389831B82DD82CC822E83CE0192
:1034A00001967FCF809590958C0D9D1DACCFF62E0B
:1034B000662309F49CCF75132EC034132CC02091C1
:1034C000AA0120FD1FC0822F82958F70D9F0D801EC
:1034D00015962C9315978F3049F08F5F982F929502
:1034E000907F822F8F70892B15968C93C8010E9434
:1034F000141586E0F801A5EAB1E001900D928A95D5
:10350000E1F793CF86E0F801A5EAB1E001900D92D2
:103510008A95E1F72DC04D875E878D859E850E9437
:103520003218811140CF8091AA0181608093AA0155
:10353000C8010E9414151CC0662309F458CF4D879A
:103540005E878D859E850E943218882309F44FCFAF
:103550002ACF811148CF0CC0243031050CF047CF61
:103560009F7009F440CFF8019581907F09F03BCF1F
:103570008F2D62960FB6F894DEBF0FBECDBFDF91E0
:10358000CF911F910F91FF90EF90DF90CF90089512
:103590001F93CF93DF93CDB7DEB72C970FB6F89478
:1035A000DEBF0FBECDBF4F83588769877A878B8771
:1035B0009C87CE0107960E940119882369F08F81AC
:1035C00098852A853B85232BF1F19F3F09F063C045
:1035D0008F3F09F060C037C086E0FE013796DE01FC
:1035E000119601900D928A95E1F76F817885EA85B1
:1035F000FB85309741F17F3F11F46F3F21F120911E
:10360000740130E0C90101968770992740917301D8
:1036100050E08417950709F447C069837A83FD83D6
:10362000EC8396E0929FD001939FB00D1124AB588C
:10363000BE4FFE01319601900D929A95E1F780936D
:1036400074010E94771816E08091730190917401C3
:103650008917C1F1189FC00111248B589E4F0E94F9
:103660000119882379F1E09173011E9FF001112463
:10367000EB58FE4F40815181628173818481958135
:103680000E9467188091730190E0019687709927D6
:1036900080937301D9CF4F81588569857A858B8551
:1036A0009C850E946718CFCF0E942E18109274013B
:1036B00010927301E5EAF1E086E0DF011D928A9540
:1036C000E9F7C1CF2C960FB6F894DEBF0FBECDBF81
:1036D000DF91CF911F910895DF92EF92FF920F93A8
:1036E0001F93CF93DF93FC01892B09F48AC0E12C4F
:1036F000F12CDD24D394EF0121968491853709F4D0
:1037000061C058F4843708F04EC0843008F06AC0B5
:103710008130D1F0823071F174C0883709F45DC016
:1037200050F4863709F455C0873709F06AC08E2DEA
:103730000E949F1D54C09CE7980F903708F061C00D
:103740008F770E949C1450C08F010E5F1F4FFE01A7
:10375000849190E2980F983050F48770FD2D01C04D
:10376000FF0F8A95EAF78F2F0E94A51D14C00E94B3
:10377000AE1313C08F010E5F1F4FFE01C49180E294
:103780008C0F883060F4C7708D2D01C0880FCA95EA
:10379000EAF70E94AB1D0E94CC1DE80125C08C2FCA
:1037A0000E949C14FACF9F012E5F3F4FFE01C491EF
:1037B000CC2369F08FE99FE00197F1F700C000008A
:1037C000C150F6CF9F012E5F3F4FFE01F490E901FB
:1037D0000BC00E948F1DE82E07C00E94A21D0E94F0
:1037E000CC1D02C00E94AE138F2D882341F0EFE95B
:1037F000FFE03197F1F700C000008150F6CFFE01E5
:103800007ACFDF91CF911F910F91FF90EF90DF90D2
:1038100008956093AF017093B0018093B1019093CC
:10382000B2010E941D1E0C941C186093AB01709392
:10383000AC018093AD019093AE010E941E1E0C94CA
:103840001C1808950C94091C0F931F930091AF014D
:103850001091B0012091B1013091B201602B712B18
:10386000822B932B1F910F910C94091C0F931F9384
:103870000091AF011091B0012091B1013091B201DE
:1038800060237123822393231F910F910C94091CB1
:103890000F931F930091AF011091B0012091B101DE
:1038A0003091B20160277127822793271F910F91D2
:1038B0000C94091C60E070E0CB010C94151C0F9374
:1038C0001F9341E050E060E070E08A019B0104C07A
:1038D000000F111F221F331F8A95D2F7C901B801AB
:1038E0001F910F910C94151C0F931F9341E050E012
:1038F00060E070E004C0440F551F661F771F8A9573
:10390000D2F78091AB019091AC01A091AD01B09143
:10391000AE018A019B01082B192B2A2B3B2BC901D5
:10392000B8011F910F910C94151C0F931F9341E048
:1039300050E060E070E004C0440F551F661F771F21
:103940008A95D2F740955095609570958091AB011E
:103950009091AC01A091AD01B091AE018A019B01A3
:10396000082319232A233B23C901B8011F910F9172
:103970000C94151C0F931F9341E050E060E070E041
:1039800004C0440F551F661F771F8A95D2F7809198
:10399000AB019091AC01A091AD01B091AE018A0153
:1039A0009B01082719272A273B27C901B8011F9126
:1039B0000F910C94151C0F931F930091AB01109164
:1039C000AC012091AD013091AE01602B712B822BA7
:1039D000932B1F910F910C94151C0F931F93009123
:1039E000AB011091AC012091AD013091AE0160238B
:1039F0007123822393231F910F910C94151C0F9315
:103A00001F930091AB011091AC012091AD01309159
:103A1000AE0160277127822793271F910F910C9485
:103A2000151C0895CF92DF92EF92FF920F931F9390
:103A3000CF93DF938C01C090AF01D090B001E090A4
:103A4000B101F090B2014091AB015091AC01609195
:103A5000AD017091AE01C42AD52AE62AF72ACFE13A
:103A6000D0E0D701C6010C2E04C0B695A795979556
:103A700087950A94D2F780FF07C0B8018C2F0E9467
:103A80002B1F8130910531F4219758F7B80180E060
:103A90000E942B1FDF91CF911F910F91FF90EF900C
:103AA000DF90CF90089520910D0130910E01F90122
:103AB00032969FEF40E05191581789F09F3F19F4DB
:103AC000511101C0942F4F5F4630A9F79F3F39F045
:103AD000F901E90FF11D97FDFA9582830895089584
:103AE00020910D0130910E01F9013296285F3F4F70
:103AF0009081981301C010823196E217F307C1F745
:103B0000089581E090E0E0910D01F0910E01E80F41
:103B1000F91F1082019688309105A9F708958091C8
:103B2000BD0108959091BD01892B8093BD01089539
:103B300080959091BD0189238093BD010895809364
:103B4000BD0108951092BD0108959091BC01892B8B
:103B50008093BC01089580959091BC018923809346
:103B6000BC0108951092BC0108958093B30108959B
:103B70001092B301089580910D0190910E01FC0106
:103B800031969C01285F3F4F80E0919191118F5FAA
:103B9000E217F307D1F70895E0910D01F0910E01BE
:103BA0008091BD018083E0910D01F0910E01908123
:103BB0008091BC01892B80838091B301882361F0BF
:103BC000E0910D01F0910E019081892B80830E947C
:103BD000BB1D81111092B30180910D0190910E01D6
:103BE0000C942412909335018093340108958295AA
:103BF000982F9C7C392F36953695282F237344E0D7
:103C0000249FC0011124932F982B292F2A7A2695BF
:103C1000892F8575880F822B08950895CF93DF93A0
:103C200000D000D01F92CDB7DEB70F900F900F904D
:103C30000F900F90DF91CF910895089508950C94FF
:103C40006C138091D301843021F11092BF0120E4E4
:103C500088E190E00FB6F894A895809360000FBEBD
:103C60002093600083B7817F846083BF83B78160C6
:103C700083BF7894889583B78E7F83BF0FB6F894FF
:103C8000A895809160008861809360001092600028
:103C90000FBE089508950895CF930E944A1E0E9472
:103CA00018080E944B1EC0E08C2F0E94160981113B
:103CB00004C0CF5FC031C1F701C081E0CF9108954A
:103CC0000C942E181F920F920FB60F9211248F93FF
:103CD0009F93AF93BF938091BF01811113C08091D7
:103CE000C0019091C101A091C201B091C301419660
:103CF000A11DB11D8093C0019093C101A093C20189
:103D0000B093C301BF91AF919F918F910F900FBE60
:103D10000F901F90189582E084BD93E095BD9AEFB7
:103D200097BD80936E0008952FB7F8948091C001DD
:103D30009091C101A091C201B091C3012FBF08951C
:103D40002FB7F8946091C0017091C1018091C201B8
:103D50009091C3012FBF0895CF92DF92EF92FF920F
:103D60000F931F932FB7F8944091C0015091C10158
:103D70006091C2017091C3012FBF6A017B01EE24E3
:103D8000FF248C0120E030E0C016D106E206F306E5
:103D900010F4415051099A01281B390BC9011F9198
:103DA0000F91FF90EF90DF90CF9008951F920F92A8
:103DB0000FB60F9211248F939F93AF93BF9380916F
:103DC000C0019091C101A091C201B091C3010196BF
:103DD000A11DB11D8093C0019093C101A093C201A8
:103DE000B093C301BF91AF919F918F910F900FBE80
:103DF0000F901F9018950E94310FF8942FEF87EACB
:103E000091E6215080409040E1F700C0000087E03B
:103E100090EBDC018093DC019093DD01A093DE0147
:103E2000B093DF019CE088E10FB6F894A8958093E9
:103E300060000FBE90936000FFCF28E0929FF001DA
:103E40001124E80FF11DE052FF4F9491892F8F70DC
:103E500092959F700895CF93C82FCB010E941D1F8C
:103E6000282F30E080E1989FA0011124422B532B92
:103E70004038510519F480E090E015C09770E92FA3
:103E8000F0E088E0C89FE00DF11D112484E0EE0F02
:103E9000FF1F8A95E1F7E20FF31FEE0FFF1FE050BF
:103EA000F84985919491CF91089580E090E008952C
:103EB00008958091C60180FF0BC06091120185E0DA
:103EC000689FB001112475956795759567952BC00E
:103ED00081FF09C06091120185E0689FB001112443
:103EE0007595679520C082FF07C06091120185E03B
:103EF000689FB001112417C09091C7019923D1F098
:103F000060911101961788F72091120185E0289F92
:103F100090011124929FA001939F500D112470E0F5
:103F2000CA010E940F276038710540F461157105C0
:103F300039F002C065E070E0862F08958FE708959C
:103F400081E008958091C60180FF08C06091100152
:103F500070E0759567957595679521C081FF06C0DE
:103F60006091100170E07595679519C082FF04C0DB
:103F70006091100170E010C09091C7019923C1F0C9
:103F800060910F019617A0F780911001899FC001E1
:103F9000112470E00E940F276038710528F4611524
:103FA000710521F0862F08958FE7089581E0089527
:103FB00061E070E0F4CF803F21F40E94591F8195A9
:103FC00004C0813F29F40E94591F8093CA010895BB
:103FD000823F21F40E94591F819504C0833F29F438
:103FE0000E94591F8093C9010895893F19F40E94C6
:103FF000A21F05C08A3F31F40E94A21F81958093C1
:10400000CB0108958B3F21F40E94A21F819504C02B
:104010008C3F29F40E94A21F8093CC010895843F15
:1040200021F48091C801816017C0853F21F48091FF
:10403000C801826011C0863F21F48091C80184606C
:104040000BC0873F21F48091C801886005C0883F7C
:1040500031F48091C80180618093C80108958D3F3B
:1040600021F48091C60181600BC08E3F21F48091C4
:10407000C601826005C08F3F29F48091C60184602B
:104080008093C6010895803F39F48091CA0187FF6B
:104090006CC01092CA0169C0813F29F48091CA01A5
:1040A0001816BCF362C09091C901823F29F497FFB2
:1040B0005CC01092C90159C0833F19F41916CCF3A2
:1040C00054C0893F41F48091CB0118160CF04DC0CB
:1040D0001092CB014AC08A3F29F48091CB0187FF1F
:1040E00044C0F6CF8B3F39F48091CC0187FF3DC0AF
:1040F0001092CC013AC08C3F29F48091CC01181663
:10410000BCF333C0843F21F48091C8018E7F17C077
:10411000853F21F48091C8018D7F11C0863F21F435
:104120008091C8018B7F0BC0873F21F48091C8012B
:10413000877F05C0883F31F48091C8018F7E8093CE
:10414000C80113C08D3F21F48091C6018E7F0BC042
:104150008E3F21F48091C6018D7F05C08F3F29F4E9
:104160008091C6018B7F8093C6018091C901811126
:104170000EC08091CA0181110AC08091CB018111CA
:1041800006C08091CC01811102C01092C701089530
:104190008091BE0183FF7EC08BEC94E00E94AD0550
:1041A0008091C8011F928F9386EC94E09F938F9328
:1041B0000E94460684EC94E00E94AD058091C901FE
:1041C000282F082E000C330B3F938F9381EC94E043
:1041D0009F938F930E9446068FEB94E00E94AD055B
:1041E0008091CA01282F082E000C330B3F938F9328
:1041F0008CEB94E09F938F930E9446068AEB94E0A9
:104200000E94AD058091CB01282F082E000C330BA6
:104210003F938F9387EB94E09F938F930E94460682
:1042200085EB94E00E94AD058091CC01282F082EEB
:10423000000C330B3F938F9382EB94E09F938F930B
:104240000E9446068FEA94E00E94AD058091C70166
:104250001F928F938CEA94E09F938F930E9446065F
:104260008AEA94E00E94AD058091C6011F928F9367
:1042700087EA94E09F938F930E94460684EA94E035
:104280000E94AD058DB79EB74C960FB6F8949EBFB1
:104290000FBE8DBF88EC91E00E946D120E94941EAB
:1042A0009093C5018093C40108951F93CF93DF932A
:1042B0008091C4019091C5010E94AC1EAC01909107
:1042C000C701992321F02091130130E006C020910D
:1042D00014018AE0289F900111244217530708F423
:1042E00085C08091C901C091CA01D091CB011091C4
:1042F000CC01811107C0C11175C0D11173C011115A
:1043000071C074C09F3F19F09F5F9093C70118164A
:1043100024F40E94591F8093C9018091C90187FF2D
:1043200005C00E94591F81958093C9011C1624F471
:104330000E94591F8093CA018091CA0187FF05C05E
:104340000E94591F81958093CA016091C90166231B
:1043500031F1C091CA01CC2311F1062E000C770B6C
:10436000880B990B0E940A2623E333E343E35FE3C0
:104370000E946E260E94D2256093C9016C2FCC0F3B
:10438000770B880B990B0E940A2623E333E343E360
:104390005FE30E946E260E94D2256093CA011D161B
:1043A00024F40E94A21F8093CB018091CB0187FF50
:1043B00005C00E94A21F81958093CB01111624F4A1
:1043C0000E94A21F8093CC018091CC0187FF05C081
:1043D0000E94A21F81958093CC01DF91CF911F9104
:1043E0000C94C8209F3F09F08FCF97CFDF91CF91DA
:1043F0001F910895E8ECF1E085E0DF011D928A95B8
:10440000E9F71092C7011092C60108958EEE96E06A
:104410000E94AD051F9281E08F931F9285E08F93DC
:1044200080EA96E09F938F930E9446060F900F902C
:104430000F900F900F900F9008958330E9F128F4BA
:10444000813061F0823009F10895853009F462C04D
:1044500008F449C0863009F474C0089580911401AD
:10446000262F30E0280F311D2F3F310524F4680F2F
:104470006093140103C08FEF8093140180911401A5
:104480001F928F9389ED95E072C080911301262FC2
:1044900030E0280F311D2F3F310524F4680F609361
:1044A000130103C08FEF80931301809113011F92BA
:1044B0008F9387EC95E05BC080911201262F30E04E
:1044C000280F311D2F3F310524F4680F609312012E
:1044D00003C08FEF80931201809112011F928F937E
:1044E00084EB95E044C080911101262F30E0280F25
:1044F000311D2F3F310524F4680F6093110103C073
:104500008FEF80931101809111011F928F938FE99A
:1045100095E02DC080911001262F30E0280F311D2D
:104520002F3F310524F4680F6093100103C08FEF13
:1045300080931001809110011F928F9386E895E07F
:1045400016C080910F01262F30E0280F311D2F3F1C
:10455000310524F4680F60930F0103C08FEF80933F
:104560000F0180910F011F928F938BE695E09F932F
:104570008F930E9446060F900F900F900F90089512
:10458000833081F128F4813059F08230D1F00895E0
:10459000853009F449C0B8F1863009F456C0089551
:1045A00080911401681720F4861B8093140102C0C7
:1045B00010921401809114011F928F938CE595E065
:1045C00054C080911301681720F4861B8093130157
:1045D00002C010921301809113011F928F938AE4FD
:1045E00095E043C080911201681720F4861B8093E8
:1045F000120102C010921201809112011F928F933A
:1046000087E395E032C080911101681720F4861B82
:104610008093110102C010921101809111011F922B
:104620008F9382E295E021C080911001681720F4F9
:10463000861B8093100102C010921001809110011E
:104640001F928F9389E095E010C080910F01681749
:1046500020F4861B80930F0102C010920F018091FD
:104660000F011F928F938EEE94E09F938F930E9481
:1046700046060F900F900F900F900895CF93C82F7C
:104680001F928F9383EF97E09F938F930E9446062C
:1046900081E090E0A0E0B0E0BC01CD0104C0660F75
:1046A000771F881F991FCA95D2F70E94221C0F906E
:1046B0000F900F900F90CF910C942E18CF938732BC
:1046C00088F58E3108F00BC18E3009F487C0D8F41C
:1046D000873009F460C08B3009F44FC0863009F090
:1046E00002C18091BE01817F8E7F8093BE0188EFE1
:1046F00097E00E94AD058BEA9AE00E94AD0581E04B
:104700008093CE0146C0863109F4B0C020F48031D8
:1047100009F47AC0E8C0893109F491C08B3109F4F9
:1047200049C0E1C0883349F150F4893209F4D5C059
:10473000853309F4D2C0873209F0D5C0CEC08334A6
:1047400009F4CBC028F48A3308F4CDC08953C8C01B
:10475000883409F0C8C00E942E188AE99AE00E94A5
:10476000AD052FEF83ED90E3215080409040E1F7BD
:1047700000C000000E94FB1E0CC08FE198E041C009
:1047800081E89AE00E94AD058091BE01816080932E
:10479000BE01C1E0ADC08091BE01C82FC17080FFD5
:1047A000EFCF8DE89AE00E94AD058091BE01817F38
:1047B0008E7F3FC09091BE0191FBCC27C0F981E074
:1047C000C827892FC0FB81F98093BE01CC2319F043
:1047D00084E79AE029C086E69AE013C09091BE0172
:1047E00092FBCC27C0F981E0C827892FC0FB82F952
:1047F0008093BE01CC2319F087E59AE015C087E4C9
:104800009AE00E94AD05C5CF9091BE0193FBCC27E5
:10481000C0F981E0C827892FC0FB83F98093BE01CE
:10482000CC2351F08BE39AE00E94AD058091BE014C
:1048300081608093BE015CC08EE29AE0E2CF8FE19E
:104840009AE00E94AD058CEF99E00E94AD0587EBE0
:1048500099E00E94AD0580E999E00E94AD058BE4E6
:1048600099E00E94AD058DE199E0CBCF8FE099E012
:104870000E94AD050E9418121F928F9385EF98E059
:104880009F938F930E94460680910C011F928F93F5
:104890008EED98E09F938F930E94460680915B0176
:1048A0001F928F938BEC98E09F938F930E94460604
:1048B0000E94A01E9F938F937F936F9384EB98E049
:1048C0009F938F930E9446068DB79EB742960FB670
:1048D000F8949EBF0FBE8DBF5CCF80E001C08D51AC
:1048E0000E943E2356CF82EB98E00E94AD05C0E0C7
:1048F0008C2FCF91089580E0089580E00895CF93A4
:10490000C82F8091CE01813069F020F0823009F407
:1049100049C040C167E08FE00E940109882309F483
:104920003FC106C067E08FE00E940109882361F063
:104930008C2F0E947B24811104C08C2F0E945E2347
:104940002FC081E090E02CC08C2F0E947D2481112B
:1049500026C0C431E1F070F4CB3081F0C031D1F425
:104960000E9406228BEE97E00E94AD0582E08093C4
:10497000CE0115C0C93259F0C83361F488EF97E011
:104980000E94AD058FEE97E00E94AD0508C0109221
:10499000CE0104C189EE97E00E94AD05FFC081E021
:1049A0008170FEC0C43228F5CE3108F0C1C0CB30D2
:1049B000A1F1D0F4C73009F0D3C08EE18093140187
:1049C00082E3809313018AE08093120184E1809353
:1049D000110188E08093100188E280930F018FE835
:1049E00096E00E94AD05BFC0C33149F1C431C1F0AA
:1049F000B7C0CB3409F4A9C028F4C93289F0C83350
:104A000061F0AEC0C13509F49EC0C23509F499C049
:104A1000CE3409F0A5C06AE09EC00E940622A3C061
:104A20008091CD01882319F01092CD019CC08CE9B2
:104A300096E00E94AD0581E08093CE01B1C086E78B
:104A400096E00E94AD0584E696E00E94AD05809157
:104A500014011F928F9381E696E09F938F930E949B
:104A600046068FE596E00E94AD058DE496E00E9433
:104A7000AD05809113011F928F938AE496E09F9376
:104A80008F930E94460688E496E00E94AD0589E374
:104A900096E00E94AD05809112011F928F9386E3EC
:104AA00096E09F938F930E94460684E396E00E94CF
:104AB000AD0583E296E00E94AD05809111011F9241
:104AC0008F9380E296E09F938F930E9446068EE13B
:104AD00096E00E94AD0589E096E00E94AD058091C8
:104AE00010011F928F9386E096E09F938F930E9410
:104AF000460684E096E00E94AD058DEE95E00E94AA
:104B0000AD0580910F011F928F938AEE95E09F93E0
:104B10008F930E94460688EE95E00E94AD058DB702
:104B20009EB748960FB6F8949EBF0FBE8DBF1BC0B0
:104B3000CE51EC2FF0E0E75DFE4F80818093CD01F8
:104B400012C061E003C061E006C06AE08091CD015F
:104B50000E941D2208C08091CD010E94C02203C086
:104B60008DE896E013C08091CD01882369F01F92F3
:104B70008F9387E896E09F938F930E9446060F904D
:104B80000F900F900F9004C084E896E00E94AD054E
:104B900081E006C01092CE0180E002C080E000CF2C
:104BA000CF9108950E94D9256894B1110C9468267C
:104BB00008950E944D2688F09F5798F0B92F9927A5
:104BC000B751B0F0E1F0660F771F881F991F1AF0F8
:104BD000BA95C9F714C0B13091F00E946726B1E0D0
:104BE00008950C946726672F782F8827B85F39F0CF
:104BF000B93FCCF3869577956795B395D9F73EF491
:104C000090958095709561957F4F8F4F9F4F089538
:104C1000E89409C097FB3EF4909580957095619556
:104C20007F4F8F4F9F4F9923A9F0F92F96E9BB270C
:104C30009395F695879577956795B795F111F8CF88
:104C4000FAF4BB0F11F460FF1BC06F5F7F4F8F4FF3
:104C50009F4F16C0882311F096E911C0772321F0E9
:104C60009EE8872F762F05C0662371F096E8862F81
:104C700070E060E02AF09A95660F771F881FDAF7D8
:104C8000880F9695879597F9089557FD9058440F8A
:104C9000551F59F05F3F71F04795880F97FB991F9B
:104CA00061F09F3F79F08795089512161306140658
:104CB000551FF2CF4695F1DF08C0161617061806E5
:104CC000991FF1CF86957105610508940895E894C0
:104CD000BB2766277727CB0197F908950E94812685
:104CE0000C94F2260E94E42638F00E94EB2620F075
:104CF000952311F00C94DB260C94E12611240C94DE
:104D000068260E94452670F3959FC1F3950F50E0E9
:104D1000551F629FF001729FBB27F00DB11D639F6D
:104D2000AA27F00DB11DAA1F649F6627B00DA11D13
:104D3000661F829F2227B00DA11D621F739FB00DB9
:104D4000A11D621F839FA00D611D221F749F332729
:104D5000A00D611D231F849F600D211D822F762FC2
:104D60006A2F11249F5750409AF0F1F088234AF09F
:104D7000EE0FFF1FBB1F661F771F881F915050400B
:104D8000A9F79E3F510580F00C94DB260C94682611
:104D90005F3FE4F3983ED4F3869577956795B79592
:104DA000F795E7959F5FC1F7FE2B880F911D9695AC
:104DB000879597F9089597F99F6780E870E060E01C
:104DC00008959FEF80EC089500240A9416161706A4
:104DD00018060906089500240A94121613061406EC
:104DE00005060895092E0394000C11F4882352F04F
:104DF000BB0F40F4BF2B11F460FF04C06F5F7F4F07
:104E00008F4F9F4F0895991B79E004C0991F961703
:104E100008F0961B881F7A95C9F78095089597FB2F
:104E2000072E16F4009407D077FD09D00E94292799
:104E300007FC05D03EF4909581959F4F089570959D
:104E400061957F4F0895EE0FFF1F0590F491E02DBF
:104E50000994AA1BBB1B51E107C0AA1FBB1FA617C1
:104E6000B70710F0A61BB70B881F991F5A95A9F713
:0E4E700080959095BC01CD010895F894FFCF78
:104E7E00FFFF830A740B510B1D0BE90A01B40128C5
:104E8E0008140A321E404D36223F04F203BC039A28
:104E9E000326033F035803710301020304050607AB
:044EAE0008090000EF
:106800000000EA44E944E2440400050006000700F1
:10681000080009000A000B000C000D000E000F001C
:1068200010001100120013001400150016001700CC
:10683000180019001A001B001C001D001E001F007C
:10684000200021002200230024002500260027002C
:10685000280029002A002B002C002D002E002F00DC
:10686000300031A132003300340035A1360037004A
:10687000380082003A003B003C003D003E003F00F3
:1068800040004100420043004400450046004700EC
:10689000480049004A004B004C004D004E004F009C
:1068A000500051005200530067005400550056003C
:1068B000580059005A005B005C005D005E005F00FC
:1068C0006000610062006300640000005700000087
:1068D000CD440000000000000000000000000000A7
:1068E0000000000000007300000000000000000035
:1068F000E000E100E200E300E400E500E600E7007C
:106900000100010001000100EA4401000100E2442D
:106910000100010001000100460001004A004B0097
:10692000010001004700480001000100E9440100A6
:106930000100010001000100010001003A003B00DC
:106940003C003D003E003F0040004100420043004B
:10695000010001004C00010001004400450052000C
:1069600049000100010050004F0001004D004E00A1
:1069700051000100010001000100010001000100BF
:1069800001000100010001000100010001000100FF
:1069900001000100010001000100010001004D00A3
:1069A0004A004E004B0001000100010001000100FF
:1069B00001000100010001000100010001000100CF
:1069C00001000100010001000100010001000100BF
:1069D00001000100010001000100010001000100AF
:1069E000010001000100010001000100010001009F
:1069F000010001000100010001000100010001008F
:00000001FF
